:020000040000FA
:060000007AEF1FF0120070
:060800007AEF1FF0120068
:06080800F8EF04F01200FD
:060818001CEF04F01200C9
:06082A000100203F000068
:08083000EC0200000A000000C8
:08083800D8CFE4FFE0CFE4FF9C
:10084000E46EDACFE4FFE2CFDAFFE9CFE4FFEACFEC
:10085000E4FFF3CFE4FFF4CFE4FFE6529EA282D0A0
:100860009E920001000ED880E655000EE7553DE24D
:100870000201EC2B000EED230001E6510201EC5DBC
:100880000001E7510201ED5930E30201EC6BED6B21
:10089000030E0001EA5D26E20001E851EA6AC80F92
:1008A000E96E020EEA2280CFEFFF0001E851EA6A0A
:1008B000CB0FE96E020EEA2281CFEFFF0001E85173
:1008C000EA6ACE0FE96E020EEA2282CFEFFF000144
:1008D000E82B030E0001E85D02E30001E86B000174
:1008E000EA2B03D00001E66BE76B0001000ED88015
:1008F000EB55000EEC5526E20001F051000822E213
:100900000201EE2B000EEF230001EB510201EE5D20
:100910000001EC510201EF5915E30201EE6BEF6BA0
:10092000030E0001EF5D0BE20001ED2B030E000151
:10093000ED5D02E30001ED6B0001EF2B03D0000140
:10094000EB6BEC6B0001F05100080CE20001F16B65
:100950000001F151040DF328C26E9E9C9F9C9D8C5A
:10096000C280C2829EAC33D09E9CC450266E26C0EC
:1009700027F0266AC35000012610246E27C025F0F8
:100980000001F151060DF3CF22F0F4CF23F0800ED9
:100990002226020E23220001ED51020D2250F324E3
:1009A000E96E2350F420EA6E24C0EEFF25C0EDFF6F
:1009B0000001F12B0001F0510001F15D02E39D9C6B
:1009C00006D00001F151040DF328C26EC282E55237
:1009D000E5CFF4FFE5CFF3FFE5CFEAFFE5CFE9FF91
:1009E000E5CFDAFFE550E5CFE0FFE5CFD8FF100017
:1009F000DACFE4FFE2CFDAFFE652E552E5CFDAFFE5
:100A00001100D9CFE6FFE1CFD9FF020EE126896AB6
:100A100092680F0EC16EC2900001F06B070EB46EAB
:100A20008A6A93688B6A9468FC0E8B16FC0E941687
:100A300094848250040B01E0010E0001606F0001FC
:100A4000E26B0001E36B0001EE6B0001ED6B000156
:100A5000EF6B0001E96B0001E86B0001EA6B00013C
:100A6000E66BE76B0001EB6BEC6BCA82CA80CA9C39
:100A7000CA9ACA88CA96FA0ECB6EDF6ADFCF14F024
:100A80000C0EE76E1418E8AE02D0E73402D0E7503F
:100A9000145C38E2010EDB6A010EDBCF14F0030EAA
:100AA000E76E1418E8AE02D0E73402D0E750145CC9
:100AB00027E2DFCF14F0156A14BE1568060E150282
:100AC000F3CF15F0060E1402F3CF14F0F4501526F0
:100AD000800E1426020E1522010EDBCF16F0176AC7
:100AE00016BE1768D8901636173614501624E96EBD
:100AF00015501720EA6EEE6AED6A010EDB2ACCD79C
:100B0000DF2ABCD7D08ECA949D829F92F28EF28C3F
:100B1000CA84020EE15C02E2E16AE552E16EE5524E
:100B2000E7CFD9FF1200D9CFE6FFE1CFD9FF080EFA
:100B3000E126010EDF6E010EDB6A020EDB6A030E98
:100B4000DB6AF8EC10F0060E0001FC5D03E36D506B
:100B5000020B01E04BD10001EA51000848E202011A
:100B6000D25145E10001E951EA6ACE0FE96E020E69
:100B7000EA22EF50E66EE66A0001E951EA6ACB0F1D
:100B8000E96E020EEA22EF50E66EE66A0001E951D4
:100B9000EA6AC80FE96E020EEA22EF50E66EE66AD4
:100BA000530E146E3E0E156E166A14C0E6FF15C085
:100BB000E6FF16C0E6FFA10EE66E000EE66EA1ECA3
:100BC0001DF0176E0B0EE15E17500001E92B030EAE
:100BD0000001E95D02E10001E96B0001EA07A10EF5
:100BE000E66E000EE66E10EC18F0E552E5520001DC
:100BF000EF51000801E3A5D00201D25101E0A1D0DC
:100C0000060EDB6A060EDBCFE9FFEA6AE9BEEA6898
:100C1000A10EE926000EEA22410EEF6E060EDB2A37
:100C2000070EDB6A0001F051F36E070EDBCFF4FF15
:100C3000F350F45C4DE2070EDBCF14F0156A14BEDE
:100C40001568060E1502F3CF15F0060E1402F3CF49
:100C500014F0F4501526800E1426020E1522000101
:100C6000EE51020D1450F324E96E1550F420EA6E93
:100C7000EECFE6FFEFCFE6FF4D0E166E3E0E176E7F
:100C8000186A16C0E6FF17C0E6FF18C0E6FF060E9A
:100C9000DBCF19F01A6A19BE1A68A10E1926000EC8
:100CA0001A2219C0E6FF1AC0E6FFA1EC1DF01B6E68
:100CB000070EE15E1B50050E146E060EDBCFE7FF3C
:100CC0001450E726060EE7CFDBFF070EDB2AAAD774
:100CD000060EDBCFE9FFEA6AE9BEEA68A10EE92663
:100CE000000EEA220A0EEF6E060EDB2A060EDBCF9E
:100CF000E9FFEA6AE9BEEA68A10EE926000EEA22E7
:100D00000D0EEF6E060EDB2A060EDBCFE9FFEA6A58
:100D1000E9BEEA68A10EE926000EEA22EF6A0001A8
:100D2000EE2B030E0001EE5D02E10001EE6B00010F
:100D3000EF07A10EE66E000EE66E10EC18F0E5521D
:100D4000E552400EE66E610EE66E000EE66ED0ECE9
:100D500017F0E552E552E552E76E010EE7CFDBFFF3
:100D60000001E16B010EDBCF14F0000EE76E1418EA
:100D7000E8AE02D0143403D0E750D880145405E212
:100D8000010EDBCFE6FF3CD8E552D950040FE66EEA
:100D9000000EDA20E66EA7D8E552E552000926E0FB
:100DA000040EDBCFE6FF1ED9E552000E0001E76E10
:100DB000E119E8AE02D0E13503D0E750D880E15523
:100DC00015E20201D25112E1E1C0A1F000010D0EC5
:100DD000A26F00010A0EA36F0001A46BA10EE66EC4
:100DE000000EE66E10EC18F0E552E552080EE15CDC
:100DF00002E2E16AE552E16EE552E7CFD9FF120067
:100E0000D9CFE6FFE1CFD9FFE652DF6AFE0EDB5015
:100E1000DF5C64E20201F35125E10D0E146EDF5038
:100E2000EA6A610FE96E000EEA22EF50145C0BE0F3
:100E30000A0E156EDF50EA6A610FE96E000EEA22B3
:100E4000EF50155C0FE10201010EF36F0001E2515A
:100E5000EA6A000FE96E020EEA220D0EEF6E000143
:100E6000E22B28D0DF50EA6A610FE96E000EEA2219
:100E7000EF500D081FE0DF50EA6A610FE96E000EC7
:100E8000EA22EF500A0816E0DF50EA6A610FE96EC5
:100E9000000EEA22EF50E66E0001E251EA6A000F0E
:100EA000E96E020EEA22E552E750EF6E0201F36BA3
:100EB0000001E22B0001E251146E156A800E141835
:100EC00002E1000E151802E10001E26B0001E3519E
:100ED0000001E25D01E102D0DF2A98D7E552E55238
:100EE000E7CFD9FF1200D9CFE6FFE1CFD9FF020E3D
:100EF000E126010EE3C0DBFF010EDB500001E25DE5
:100F00000BE1FD0EDBCFE9FFFE0EDBCFEAFFEF6A60
:100F10000001616B000E5AD0DF6ADF50146E156A53
:100F2000D890155004E6800E145C000E155843E26C
:100F3000010EDB50EA6A000FE96E020EEA22EF5062
:100F4000E66EDF50EA6A610FE96E000EEA22E552B2
:100F5000E750EF6E010EDB2A010EDB50146E156AAE
:100F6000800E141802E1000E151802E1010EDB6A72
:100F70000D0E146EDF50EA6A610FE96E000EEA2270
:100F8000EF50145C10E1DF28E66EFD0EDBCFE9FFC9
:100F9000FE0EDBCFEAFFE552E750EF6E010EDBCF2E
:100FA000E3F0010E13D0010EDB500001E25D01E120
:100FB00002D0DF2AB2D7FD0EDBCFE9FFFE0EDBCF7A
:100FC000EAFFEF6A0001616B000E00D0146E020EA2
:100FD000E15C02E2E16AE552E16E1450E552E7CFCE
:100FE000D9FF1200D9CFE6FFE1CFD9FFFE0EDB0417
:100FF0000CE0FE0EDB5002080CE22C0E0001625DDC
:1010000008E02C0E0001635D04E000012C0EE16F8E
:1010100087D0FE0EDB04EA6A610FE96E000EEA2259
:10102000EF500D0804E00001210EE16F79D00001BE
:1010300061514D0A5FE01D0A46E0040A32E0150ADC
:101040002EE0170A2AE01F0A26E0060A22E00C0A10
:101050000EE0110A01E05FD000016251580A01E080
:1010600003D098EC0EF002D05FD800D059D0000128
:101070006251580A05E0740A01E005D000D908D091
:1010800099EC0EF005D000013F0EE16F49D000D081
:1010900047D0A3D945D01EDA43D046DA41D050DA42
:1010A0003FD000016251580A05E0740A01E005D002
:1010B00056D808D097EC0EF005D000013F0EE16F36
:1010C0002FD000D02DD000016251440A0BE00B0A52
:1010D00006E0060A01E008D0F9EC0CF00AD0B1EC09
:1010E0000DF007D0A0DB05D000013F0EE16F18D056
:1010F00000D016D000016251570A05E0050A01E050
:1011000004D023DB07D0AFDA05D000013F0EE16F3A
:1011100007D000D005D000013F0EE16F01D000D014
:10112000E552E7CFD9FF12006CDC0201D25116E183
:1011300000014F0EA16F00014B0EA26F00010A0EBD
:10114000A36F00010D0EA46F0001A56BA10EE66E4A
:10115000000EE66E10EC18F0E552E5521200D9CF01
:10116000E6FFE1CFD9FF020EE126010EDF6E010E90
:10117000DB6A030EE66ED9CFE6FFDACFE6FFCDECF1
:101180000EF0E552E552E55207C0E4F008C0E5F084
:10119000010EE66ED9CFE6FFDACFE6FFCDEC0EF01A
:1011A000E552E552E552010E07C0DBFF0001E151B7
:1011B00001E05BD0DF50EA6A610FE96E000EEA22BF
:1011C000EF500D0807E00001E15104E10001230E9A
:1011D000E16F4BD0010EDB5018E10001E451E51145
:1011E00004E10001E66BE76B0FD000010A0EE45D3D
:1011F000000EE55904E20A0E0001E46FE56BCA84B3
:10120000E4C0E6F0E5C0E7F017D00001E451E511D5
:1012100004E10001EB6BEC6B0FD000010A0EE45D02
:10122000000EE55904E20A0E0001E46FE56BCA8482
:10123000E4C0EBF0E5C0ECF00201D25116E1000190
:101240004F0EA16F00014B0EA26F00010A0EA36F9B
:1012500000010D0EA46F0001A56BA10EE66E000E3D
:10126000E66E10EC18F0E552E552020EE15C02E287
:10127000E16AE552E16EE552E7CFD9FF1200D9CF1E
:10128000E6FFE1CFD9FF050EE126010EF36E040E55
:10129000F3CFDBFF010EE66ED950040FE66E000EB1
:1012A000DA20E66ECDEC0EF0E552E552E55207503D
:1012B000DF6E010EE66ED950040FE66E000EDA20E6
:1012C000E66ECDEC0EF0E552E552E552010E07C098
:1012D000DBFF010EE66ED950040FE66E000EDA2039
:1012E000E66ECDEC0EF0E552E552E552020E07C077
:1012F000DBFF010EE66ED950040FE66E000EDA2019
:10130000E66ECDEC0EF0E552E552E552030E07C055
:10131000DBFF0001E15101E056D0040EDB50EA6A28
:10132000610FE96E000EEA22EF500D0807E00001A0
:10133000E15104E10001230EE16F45D00201D251D9
:1013400016E100014F0EA16F00014B0EA26F0001CC
:101350000A0EA36F00010D0EA46F0001A56BA10E74
:10136000E66E000EE66E10EC18F0E552E552DF5026
:10137000926E010EDB50936E020EDB50946E030EE4
:10138000DB500C0805E20C0EF36E030EF3CFDBFF0F
:10139000030EDB5006E10F0EC16EC2900001F06B30
:1013A00012D00001F06BC26A030EDBCFE6FF0F0E16
:1013B000E552D880E754C16EBE0EC06EC280030EE7
:1013C000DBCFF0F0CA84050EE15C02E2E16AE5528F
:1013D000E16EE552E7CFD9FF1200D9CFE6FFE1CFAA
:1013E000D9FF040EE126010EF36E030EF3CFDBFFEF
:1013F000010EE66ED950030FE66E000EDA20E66E9F
:10140000CDEC0EF0E552E552E5520750DF6E010ECD
:10141000E66ED950030FE66E000EDA20E66ECDECD4
:101420000EF0E552E552E552010E07C0DBFF010E5A
:10143000E66ED950030FE66E000EDA20E66ECDECB4
:101440000EF0E552E552E552020E07C0DBFF000147
:10145000E15101E035D0030EDB50EA6A610FE96E1D
:10146000000EEA22EF500D0807E00001E15104E10F
:101470000001230EE16F24D00001E15108E1DF50AB
:10148000896E010EDB508A6E020EDB508B6E0201FC
:10149000D25116E100014F0EA16F00014B0EA26F59
:1014A00000010A0EA36F00010D0EA46F0001A56BD1
:1014B000A10EE66E000EE66E10EC18F0E552E55255
:1014C000040EE15C02E2E16AE552E16EE552E7CF2B
:1014D000D9FF12000201D25126E18250E66EE66A7F
:1014E0008150E66EE66A8050E66EE66A530E146E30
:1014F0003E0E156E166A14C0E6FF15C0E6FF16C054
:10150000E6FFA10EE66E000EE66EA1EC1DF0176E72
:101510000B0EE15E1750A10EE66E000EE66E10ECAB
:1015200018F0E552E55212000201D25108E1DA0E3C
:10153000E66E3E0EE66E4EEC18F0E552E5521200F5
:10154000D9CFE6FFE1CFD9FF020EE126DF6A010E17
:10155000DB6A0201D25101E07CD0DFCFE9FFEA6A09
:10156000E9BEEA68A10EE926000EEA22410EEF6EFE
:10157000DF2A010EDB6A0001F051F36E010EDBCFB2
:10158000F4FFF350F45C3BE2010EDBCFE9FFEA6AC3
:10159000E9BEEA68060EEA02F3CFEAFF060EE902A8
:1015A000F3CFE9FFF450EA26800EE926020EEA2284
:1015B000EECFE6FFEFCFE6FF4D0E146E3E0E156E3A
:1015C000166A14C0E6FF15C0E6FF16C0E6FFDFCFBF
:1015D00017F0186A17BE1868A10E1726000E1822F9
:1015E00017C0E6FF18C0E6FFA1EC1DF0196E070E4C
:1015F000E15E1950050EDF26010EDB2ABCD7DFCFD6
:10160000E9FFEA6AE9BEEA68A10EE926000EEA22CD
:101610000A0EEF6EDF2ADFCFE9FFEA6AE9BEEA6869
:10162000A10EE926000EEA220D0EEF6EDF2ADFCFB3
:10163000E9FFEA6AE9BEEA68A10EE926000EEA229D
:10164000EF6AA10EE66E000EE66E10EC18F0E552A1
:10165000E552020EE15C02E2E16AE552E16EE5521A
:10166000E7CFD9FF1200D9CFE6FFE1CFD9FF040EB3
:10167000E126020EF36E030EF3CFDBFF030EE66EE0
:10168000D950030FE66E000EDA20E66E86DBE552D7
:10169000E552E55207C0DEFF08C0DDFF010EE66E31
:1016A000D950030FE66E000EDA20E66E76DBE552C7
:1016B000E552E552020E07C0DBFF0001E15101E0F7
:1016C0003AD0030EDB50EA6A610FE96E000EEA229F
:1016D000EF500D0807E00001E15104E10001230E85
:1016E000E16F29D0DECF14F0DDCF15F0000E145CD1
:1016F000100E155807E2DECFE9FFDDCFEAFF020E3C
:10170000DBCFEFFF0201D25116E100014F0EA16FB6
:1017100000014B0EA26F00010A0EA36F00010D0E17
:10172000A46F0001A56BA10EE66E000EE66E10EC34
:1017300018F0E552E552040EE15C02E2E16AE5527E
:10174000E16EE552E7CFD9FF1200D9CFE6FFE1CF36
:10175000D9FF040EE126020EF36E030EF3CFDBFF7A
:10176000030EE66ED950030FE66E000EDA20E66E29
:1017700014DBE552E552E55207C0DEFF08C0DDFF8D
:101780000001E15101E045D0030EDB50EA6A610F30
:10179000E96E000EEA22EF500D0807E00001E1516A
:1017A00004E10001230EE16F34D0DECF14F0DDCF71
:1017B00015F0000E145C100E155807E2DECFE9FF9D
:1017C000DDCFEAFF020EEFCFDBFF0201D25121E1B4
:1017D000020EDBCFE6FFE66A430E146E3E0E156E78
:1017E000166A14C0E6FF15C0E6FF16C0E6FFA10E9C
:1017F000E66E000EE66EA1EC1DF0176E070EE15EC0
:101800001750A10EE66E000EE66E10EC18F0E552D1
:10181000E552040EE15C02E2E16AE552E16EE55256
:10182000E7CFD9FF1200D9CFE6FFE1CFD9FF040EF1
:10183000E126020EF36E030EF3CFDBFF040EE66E1D
:10184000D950030FE66E000EDA20E66EA6DAE552F6
:10185000E552E5520750DF6E010EE66ED950030FD8
:10186000E66E000EDA20E66E98DAE552E552E552B1
:10187000010E07C0DBFF010EE66ED950030FE66EC6
:10188000000EDA20E66E89DAE552E552E552020EE4
:1018900007C0DBFF0001E15101E0A1D0030EDB50E6
:1018A000EA6A610FE96E000EEA22EF500D0807E0C8
:1018B0000001E15104E10001230EE16F90D0020E1E
:1018C000DB50010804E200012A0EE16F88D0010E0E
:1018D000DB50070804E200012A0EE16F80D0410EC0
:1018E000146EDF50145C1CE1020EDB500DE1010EA2
:1018F000F36E010EDB5004E0D890F336E806FCE10D
:10190000F350E81C92160BD0010EF36E010EDB5063
:1019100004E0D890F336E806FCE1F350921246D08A
:10192000420E146EDF50145C1CE1020EDB500DE120
:10193000010EF36E010EDB5004E0D890F336E8069A
:10194000FCE1F350E81C93160BD0010EF36E010E70
:10195000DB5004E0D890F336E806FCE1F350931234
:1019600025D0430E146EDF50145C1CE1020EDB50D8
:101970000DE1010EF36E010EDB5004E0D890F3365A
:10198000E806FCE1F350E81C94160BD0010EF36E50
:10199000010EDB5004E0D890F336E806FCE1F3508A
:1019A000941204D000012A0EE16F19D00201D25125
:1019B00016E100014F0EA16F00014B0EA26F000156
:1019C0000A0EA36F00010D0EA46F0001A56BA10EFE
:1019D000E66E000EE66E10EC18F0E552E552040ECD
:1019E000E15C02E2E16AE552E16EE552E7CFD9FF40
:1019F0001200D9CFE6FFE1CFD9FF040EE126020E97
:101A0000F36E020EF3CFDBFF030EDB6A040EE66E0D
:101A1000D950020FE66E000EDA20E66EBED9E5520E
:101A2000E552E5520750DF6E010EE66ED950020F07
:101A3000E66E000EDA20E66EB0D9E552E552E552C8
:101A4000010E07C0DBFF0001E15101E080D0020E72
:101A5000DB50EA6A610FE96E000EEA22EF500D08D2
:101A600007E00001E15104E10001230EE16F6FD0B6
:101A7000010EDB50070804E200012A0EE16F67D077
:101A8000410E146EDF50145C10E1010EF36E010E76
:101A9000DB5004E0D890F336E806FCE1F350801404
:101AA000E76E030EE7CFDBFF2ED0420E146EDF5041
:101AB000145C10E1010EF36E010EDB5004E0D890CF
:101AC000F336E806FCE1F3508114E76E030EE7CF2E
:101AD000DBFF19D0430E146EDF50145C10E1010ED1
:101AE000F36E010EDB5004E0D890F336E806FCE11B
:101AF000F3508214E76E030EE7CFDBFF04D0000142
:101B00002A0EE16F24D00201D25121E1030EDBCF76
:101B1000E6FFE66A3A0E146E3E0E156E166A14C0A3
:101B2000E6FF15C0E6FF16C0E6FFA10EE66E000E4A
:101B3000E66EA1EC1DF0176E070EE15E1750A10EC8
:101B4000E66E000EE66E10EC18F0E552E552040E5B
:101B5000E15C02E2E16AE552E16EE552E7CFD9FFCE
:101B60001200D9CFE6FFE1CFD9FF040EE126020E25
:101B7000F36E030EF3CFDBFF040EE66ED950030FB6
:101B8000E66E000EDA20E66E08D9E552E552E5521F
:101B90000750DF6E010EE66ED950030FE66E000EA1
:101BA000DA20E66EFAD8E552E552E552010E07C09A
:101BB000DBFF010EE66ED950030FE66E000EDA2051
:101BC000E66EEBD8E552E552E552020E07C0DBFFA8
:101BD0000001E15101E0A1D0030EDB50EA6A610F80
:101BE000E96E000EEA22EF500D0807E00001E15116
:101BF00004E10001230EE16F90D0020EDB500108DA
:101C000004E200012A0EE16F88D0010EDB500708C4
:101C100004E200012A0EE16F80D0410E146EDF5005
:101C2000145C1CE1020EDB500DE1010EF36E010E9F
:101C3000DB5004E0D890F336E806FCE1F350E81CF2
:101C400089160BD0010EF36E010EDB5004E0D89024
:101C5000F336E806FCE1F350891246D0420E146ECA
:101C6000DF50145C1CE1020EDB500DE1010EF36E3F
:101C7000010EDB5004E0D890F336E806FCE1F350A7
:101C8000E81C8A160BD0010EF36E010EDB5004E047
:101C9000D890F336E806FCE1F3508A1225D0430EC3
:101CA000146EDF50145C1CE1020EDB500DE1010EDE
:101CB000F36E010EDB5004E0D890F336E806FCE149
:101CC000F350E81C8B160BD0010EF36E010EDB50A7
:101CD00004E0D890F336E806FCE1F3508B1204D010
:101CE00000012A0EE16F19D00201D25116E1000164
:101CF0004F0EA16F00014B0EA26F00010A0EA36FE1
:101D000000010D0EA46F0001A56BA10EE66E000E82
:101D1000E66E10EC18F0E552E552040EE15C02E2CA
:101D2000E16AE552E16EE552E7CFD9FF12001200F9
:101D300012000201D25116E100014F0EA16F000105
:101D40004B0EA26F00010A0EA36F00010D0EA46FCF
:101D50000001A56BA10EE66E000EE66E10EC18F009
:101D6000E552E55212000201D25116E100014F0E78
:101D7000A16F00014B0EA26F00010A0EA36F0001BC
:101D80000D0EA46F0001A56BA10EE66E000EE66EAF
:101D900010EC18F0E552E5521200D9CFE6FFE1CF82
:101DA000D9FF040EE126030EDB6A0001E15104E0D5
:101DB000076A086A096A69D1FD0EDBCFE9FFFE0EEA
:101DC000DBCFEAFFEF50EA6A610FE96E000EEA220C
:101DD000EF502C0807E000015E0EE16F076A086A09
:101DE000096A53D1FD0EDBCFE9FFFE0EDBCFEAFF20
:101DF000EF2A2D0E146EFD0EDBCFE9FFFE0EDBCFBA
:101E0000EAFFEF50EA6A610FE96E000EEA22EF5036
:101E1000145C23E1040E156EFC0EDB50155C1DE016
:101E2000FC0EDB0406E0030E146EFC0EDB50145CAB
:101E300008E100017C0EE16F076A086A096A25D192
:101E40000CD0010EF36E030EF3CFDBFFFD0EDBCFE4
:101E5000E9FFFE0EDBCFEAFFEF2A040E146EFC0E44
:101E6000DB50145C12E0050EE66ED9CFE6FFDACF48
:101E7000E6FFFD0EDBCFE6FFFE0EDBCFE6FF0FD960
:101E8000146E050EE15E14501FD0FD0EDBCFE9FF8E
:101E9000FE0EDBCFEAFFEF50EA6A610FE96E000E3B
:101EA000EA22EFCF14F0156A166A14C0DFFF010EA4
:101EB00015C0DBFF020E16C0DBFFFD0EDBCFE9FF16
:101EC000FE0EDBCFEAFFEF2A030EDB5021E0DFCF6F
:101ED00014F0010EDBCF15F0020EDBCF16F00C680C
:101EE0000D680E6814C007F015C008F016C009F0A0
:101EF000C4EC1CF004C014F005C015F006C016F0C8
:101F000014C0DFFF010E15C0DBFF020E16C0DBFFA1
:101F1000FC0EDB5026E1DFCF14F0010EDBCF15F015
:101F2000020EDBCF16F01634000E161807E6D88026
:101F30007F0E1454000E1554000E165401E28CD07E
:101F4000D9CFE9FFDACFEAFF020ED880EB50FF0AC3
:101F500006E6800EEE5CFF0EEE58FF0EEF5801E233
:101F60007BD0FC0EDB0424E1DFCF17F0010EDBCFCA
:101F700018F0020EDBCF19F01934000E191807E61D
:101F8000D880FF0E1754000E1854000E195464E345
:101F9000D9CFE9FFDACFEAFF020ED890EB50000A62
:101FA00006E6000EEE5C000EEE58000EEF5854E30D
:101FB000020E1A6EFC0EDB501A5C24E1DFCF1BF020
:101FC000010EDBCF1CF0020EDBCF1DF01D34000E26
:101FD0001D1807E6D880FF0E1B547F0E1C54000E00
:101FE0001D543AE3D9CFE9FFDACFEAFF020ED880D9
:101FF000EB50FF0A06E6000EEE5C800EEE58FF0E78
:10200000EF582AE3030E1E6EFC0EDB501E5C2EE121
:10201000DFCF1FF0010EDBCF20F0020EDBCF21F06F
:102020002134000E211807E6D880FF0E1F54FF0E42
:102030002054000E215410E3D9CFE9FFDACFEAFF94
:10204000020ED890EB50000A06E6000EEE5C000E81
:10205000EE58000EEF580AE20001E15107E10001DD
:102060007E0EE16F076A086A096A0FD0DFCF14F0AD
:10207000010EDBCF15F0020EDBCF16F014C007F017
:1020800015C008F016C009F000D0040EE15C02E2B1
:10209000E16AE552E16EE552E7CFD9FF1200D9CFF0
:1020A000E6FFE1CFD9FF020EE126FB0EDBCFE9FF11
:1020B000FC0EDBCFEAFFEE6AEE6AEE6A010EDB6A27
:1020C000FA0EDB50F36E010EDBCFF4FFF350F45C3D
:1020D00059E2FD0EDBCFE9FFFE0EDBCFEAFFEF504A
:1020E000EA6A610FE96E000EEA22EFCFDFFF300EE1
:1020F000DF5C43E3DF50390840E3FB0EDBCFE9FF51
:10210000FC0EDBCFEAFFEECF17F0EECF18F0EFCFEB
:1021100019F00A0E0C6E0D6A0E6A17C007F018C08F
:1021200008F019C009F0C4EC1CF004C017F005C099
:1021300018F006C019F0300EDF5C1A6E1B6A1C6ABC
:1021400017501A24146E18501B20156E19501C209D
:10215000166EFB0EDBCFE9FFFC0EDBCFEAFF14C0EF
:10216000EEFF15C0EEFF16C0EEFFFD0EDBCFE9FF60
:10217000FE0EDBCFEAFFEF2A02D0000E05D0010EE3
:10218000DB2A9ED7010E00D0146E020EE15C02E243
:10219000E16AE552E16E1450E552E7CFD9FF120033
:1021A0000001E15124E10201D25121E10001EA5193
:1021B000E66EE66A2E0E146E3E0E156E166A14C09A
:1021C000E6FF15C0E6FF16C0E6FFA10EE66E000EA4
:1021D000E66EA1EC1DF0176E070EE15E1750A10E22
:1021E000E66E000EE66E10EC18F0E552E5521200B5
:1021F0000201F451F51105E10201500EF46FC30E16
:10220000F56F0201F407000EF55B0001FC5108E0D8
:10221000010E146E6D50020B01E0010E145C02E120
:102220008B901AD00001FC050CE0020E0001FC5D51
:1022300008E0030E0001FC5D04E0050E0001FC5DFA
:1022400002E18B8009D0060E0001FC5D05E1020170
:10225000F451F51101E18B70120082B403D0010E2C
:0A22600003D002D0000E00D01200DF
:06226A0071EC16F0FB0E02
:10227000DBCFF3FFDB06F35000090AE0BFEC16F0FA
:10228000FA0E2AEC17F0F3E1151CF1E1010E01D072
:10229000000EA0EF16F071EC16F03B0EE12402E305
:1022A000E168E652E16E010EDB6A020EDB6AF90EAE
:1022B000DBCFF6FFFA0EDBCFF7FFFB0EDBCFF8FF2D
:1022C0000800F550DF6EDF5002E1C4EF15F0250E77
:1022D000DF5C02E0B7EF15F0030EDB6A040EDB6A89
:1022E000050EDB6A060EDB6A070EDB6AD9EC15F019
:1022F0002D0EDF5C0CE02B0EDF5C09E0200EDF5CB6
:1023000006E0230EDF5C03E0300EDF5C1AE1DF50F5
:10231000300A14E0130A0FE0030A0AE00B0A05E092
:10232000060AE4E1030EDB80E1D7030EDB82DED791
:10233000030EDB84DBD7030EDB86D8D7030EDB88E6
:10234000D5D72A0EDF5C1BE1D5EC15F023EC16F097
:1023500010E0030EDB8008680968130EDBCF0DF078
:10236000140EDBCF0EF00DEC1DF0040E06C0DBFFEB
:1023700003D0130E0CEC16F0D9EC15F00BD0090EAF
:10238000DB6A7AEC16F003E0EEEC16F0FAD7090EF1
:102390000CEC16F0030EDBB0DB982E0EDF5C1BE1BD
:1023A000D9EC15F02A0EDF5C0BE1D5EC15F023EC2F
:1023B00016F003E1130E5EEC16F0D9EC15F00BD01D
:1023C000090EDB6A7AEC16F003E0EEEC16F0FAD7B1
:1023D000090E5EEC16F0680EDF5C07E1D9EC15F033
:1023E000680EDF5C1DE1030E18D0740EDF5C17E091
:1023F0007A0EDF5C14E0480EDF5C06E0540EDF5C12
:1024000003E05A0EDF5C02E1020E07D06C0EDF5CC7
:1024100003E06A0EDF5C04E1010EB1EC16F0C9DBEB
:10242000DF506E0A01E17FD31E0A01E192D1200A3A
:1024300001E18FD13F0A01E149D11A0A01E146D1F8
:102440000D0A01E143D1200A01E140D13A0A01E13C
:102450003DD1200A01E13AD1260A01E135D10D0A28
:1024600001E132D11A0A01E1D9D0200A4AE0300A4A
:102470001FE0460A0EE0250A01E083D3D950F90F88
:10248000E96EFF0EDA20EA6E010EEE5E000EEE5AE5
:10249000EE5ABFEC16F0250EE66E95DB03E1151C37
:1024A00001E169D3BBEC16F001E26BD3DB2A69D3FF
:1024B000080EDB6A040EDB50010806E2040EDB04A2
:1024C00083EC16F0DB508BDB080EDB5009E0030ECB
:1024D000DB50010B05E172DB01E04DD3080EDB6A36
:1024E00064DBEFCFDFFF33EC17F003E1151C01E1F4
:1024F00042D3BBEC16F001E3DB2A60DB01E141D300
:102500003AD3070EDB5002080FE1FFEC16F0030E82
:10251000C6EC16F00E0EEECFDBFF0F0EEECFDBFF9C
:10252000100EEECFDBFF20D0F70EDBCF17F0F80E4A
:10253000DBCF18F0020E175E000E185AF70E17C008
:10254000DBFFF80E18C0DBFF17C0E9FF18C0EAFF79
:10255000B6EC16F0166A0E0E14C0DBFF0F0E15C097
:10256000DBFF100E16C0DBFF0E0EDBCFE6FF0F0EFB
:10257000DBCFE6FF100EDBCFE6FFCEEC1EF0E55220
:10258000E552E552130E07C0DBFF140E08C0DBFF57
:10259000060EDB5005E0130EFAEC16F001E26ADBE2
:1025A0001EEC17F002E2130E37DBE1EC16F006E04A
:1025B000040EFAEC16F002E2050E2EDB030EDBB081
:1025C00005D0FCDA01E0D7D2080EDB6A090EDB6A1F
:1025D0000E0EDBCFF6FF0F0EDBCFF7FF100EDBCFBB
:1025E000F8FF0800F550DF6EDF5014E024EC17F020
:1025F00011E233EC17F003E1151C01E1BCD2BBDBA7
:1026000001E3DB2A090EDB2AD9500E0FE96E000E1A
:10261000CBDBE7D7D3DA01E1B4D2ADD2C6DA110E03
:10262000EECFDBFF120EEDCFDBFF110EDBCFE6FFAF
:10263000120EDBCFE6FFC0EC1EF0E552E552130EA2
:10264000F3CFDBFF140EF4CFDBFF060EDB5004E00C
:10265000130ED0DB01E20EDB1EEC17F002E2130ECC
:10266000DBDAAFDB05E0040EC5DB02E2050ED4DAEF
:10267000030EDBB005D0A2DA01E07DD2080EDB6AE2
:10268000090EDB6A110EDBCFE9FF120EDBCFEAFF8A
:10269000EFCFDFFFDF5014E0D7DB12E2E4DB03E132
:1026A000151C01E168D267DB01E3DB2A090EDB2A96
:1026B000110EDB2ADBCFE9FF120EE8E3DB2AE6D7B7
:1026C0007DDA01E15ED257D2030EDB8E070EDB040A
:1026D00010E195DB040E5ADB0A0EEECFDBFF0B0E8A
:1026E000EECFDBFF0C0EEECFDBFF0D0EEECFDBFFF0
:1026F0006CD0070EDB5003082CE1030EDBAE0DD0CF
:10270000B2DA020E76DAEFCF14F0156A166A176A9B
:1027100014AE39D01568166835D0F70EDBCF15F03A
:10272000F80EDBCF16F0020E155E000E165AF70EED
:1027300015C0DBFFF80E16C0DBFF15C0E9FF16C0A1
:10274000EAFFEFCF14F00A0E14C0DBFF0B0EDB6ABA
:1027500038D0070EDB50020809E1030EDBAE04D0CF
:1027600059DB16AE10D00ED055DB0DD0030EDBAE0C
:1027700012D079DA020E3DDAF9DA166A176A15AE66
:1027800002D016681768E2DA0C0E16C0DBFF0D0ED9
:1027900017C0DBFF1AD0F70EDBCF16F0F80EDBCF39
:1027A00017F0020E165E000E175AF70E16C0DBFF6A
:1027B000F80E17C0DBFF16C0E9FF17C0EAFFD6DA34
:1027C000C5DA0C0EDB6A0D0EDB6A060EDB5005E186
:1027D000010EF36E050EF3CFDBFF150EDB6A160E4E
:1027E000DB6AD950370F146E000EDA20156E390EE1
:1027F00014C0DBFF3A0E15C0DBFF380EDB6A080E93
:10280000DB6A0A0EAEDADF50780A12E0200A10E026
:10281000280A0CE0200A0AE03F0A06E00D0A02E05E
:10282000200A08E1020E05D0080E03D0080EDF26AC
:10283000100E97DA030EDBBE02D0DB92DB94DB5086
:10284000800B24E08ADAD890030EEB50000A08E6E9
:10285000000EEE5C000EEE58000EEE58000EEE5824
:1028600015E213DA0B680C680D680E6888EC1EF030
:102870000A0E02C0DBFF0B0E03C0DBFF0C0E04C010
:10288000DBFF0D0E05C0DBFF2D0E08D0030EDBA213
:1028900002D02B0E03D0DBA408D0200EF36E170E4F
:1028A000F3CFDBFF150EDB2A02D0170EDB6A050E15
:1028B000DB5003E1B7D901E189D00C0E146E3F0E55
:1028C000156E000E166E070EDBCF17F0186A196A28
:1028D0001A6A17C00BF018C00CF019C00DF01AC01E
:1028E0000EF0D3D9F3EC1EF014500224F36E155001
:1028F0000320F46E16500420F86EF4CFF7FFF3CFE8
:10290000F6FF0800090EF5CFDBFF580EDF5C0FE184
:10291000610EF36E090E7BD90AE3200E146E090EC8
:10292000DBCFE7FF1450E75E090EE7CFDBFF070EB2
:10293000DBCF14F0156A166A176A0FDA14C00BF0B1
:1029400015C00CF016C00DF017C00EF0EECF06F05B
:10295000EECF07F0EECF08F0EFCF09F0F3EC1EF06A
:1029600009C0EDFF08C0EDFF07C0EDFF06C0EFFF97
:10297000390EDBCFE9FFDB063A0EDBCFEAFF01E2DF
:10298000DB06090EDBCFEFFF150EDB2A4BD995E1F5
:10299000030EDBA61DD06F0EDF5C06E1C1D918E384
:1029A000150EDB285BDA14D0780EDF5C09E0580ED8
:1029B000DF5C06E0620EDF5C03E0420EDF5C08E1F4
:1029C000020EF36E160EF3CFDBFF02D0150EDB6A9C
:1029D000030EDB50100B0EE0040EDBCF14F0050EDF
:1029E000DB50D880145406E2060EDB5003E1040EDF
:1029F000DB5034DA95D90AE2050EDBCFE7FF150E7E
:102A0000DB50E75E050EE7CFDBFF02D0050EDB6A89
:102A1000040EDBCF14F0160E45D9D880145414E2FE
:102A2000160EDBCFE6FF150EDBCFE6FF040EDBCF85
:102A3000E6FF050EDB50E552E75CE552D880E7542F
:102A4000E552D880E7545FD9030EDB50010B0BE150
:102A5000080EDB5008E0B2D801E08DD0080EDB5044
:102A6000BED8080EDB6A170EDB5007E088D9170EB8
:102A7000F1D903E1151C01E17ED0160EDB5016E002
:102A80007ED9300EE66E9FD802E1151C74E077D92E
:102A9000DFCFE6FF46EC1EF0E552E552E552F4CFFB
:102AA00015F00001F31C02E1151C65E0050EDBCFFB
:102AB00014F0160EDB50D880145409E2050EDBCF5B
:102AC000E7FF160EDB50E75E050EE7CFDBFF300EAB
:102AD000E66E050ECBD94FE1390EDB2ADBCFE9FFDD
:102AE0003A0E01E3DB2ADBCFEAFF090EEFCFDBFF73
:102AF000DB500EE044D9090EADD902E1151C3BE0D4
:102B0000390EDB2ADBCFE9FF3A0EEDE3DB2AEBD708
:102B100055D831E1160EDBCFE6FF080EC3D8E552DB
:102B2000E7245DD82ED0070EDB50030A1CE0010A13
:102B300014E0030A07E07BD9DBCFEEFF020EDBCF08
:102B4000EDFF1FD0F5D8196A17AE02D018681968C2
:102B50002CD8BCD819C0EEFF14D0EAD817BE18681C
:102B600024D8B4D80ED063D9DBCFEFFF0AD07BD9FD
:102B700005E1151C03E1F368F46810D0FCD801E30B
:102B8000DB2A79D960EF11F0010EDBCF14F0020ED1
:102B9000DBCF15F014C0F3FF15C0F4FF3B0EE15C72
:102BA00002E2E16AE552E16ECBD029D9020EC6EF0E
:102BB00016F061D90800F550DF6E1200200EE66EA7
:102BC000080E36EF17F046EC1EF0E552E552E552DE
:102BD000F3CF14F0F4CF15F00001F31C1200146EC3
:102BE000156AD950010F4DD91450EE261550ED221B
:102BF0001200185E000E195AF70E18C0DBFFF80E0F
:102C000019C0DBFF18C0E9FF19C0EAFF1200DBCFD3
:102C1000F4FFF350F45C1200DB50E76E040EE7CFD4
:102C2000DBFF12000A0EDBCF14F00B0EDBCF15F02A
:102C30000C0EDBCF16F00D0EDBCF17F01450151075
:102C4000161017101200130EEECFDBFF140EEDCF8F
:102C5000DBFF130EDBCF14F0140EDBCF15F00001F9
:102C6000800E15141200F70EDBCF18F0F80EDBCF34
:102C700019F01200050EDB50E66ED950130F01D982
:102C8000E552E750EE6EED6A12000A0EDBCF06F059
:102C90000B0EDBCF07F00C0EDBCF08F00D0EDBCFF9
:102CA00009F01200DBCFE6FF150EDBCFE6FF050EC5
:102CB000DB50E552E724E552E7241200DB50CED882
:102CC000010EF36E060EF3CFDBFF1200EE50EFCFD6
:102CD000EAFFE96E16C0EEFF17C0EEFF18C0EEFF68
:102CE0001200D9CFE6FFDACFE6FFE1CFD9FFE2CF7E
:102CF000DAFF1200DFCFE6FFE66A4DEC1FF0E55287
:102D0000E552F3501200E76E080EE7CFDBFF12002A
:102D1000EECF14F0EECF15F0EFCF16F0176A1200D9
:102D2000050EDBCF14F0150EDB50D88014541200C2
:102D3000010EDBCF16F0020EDBCF17F0186A12007F
:102D4000E552E5CFDAFFE7CFD9FF12000A0E14C033
:102D5000DBFF0B0E15C0DBFF1200D9500A0F41EF4D
:102D600017F0F36E070EF3CFDBFF1200EECF14F077
:102D7000EFCF15F01200010EDB2A020E1200FC0E3E
:102D8000DBCFE6FFFD0EDBCFE6FF1200145E000E88
:102D9000155AF70E14C0DBFFF80E15C0DBFF14C088
:102DA000E9FF15C0EAFF1200DA20EA6EEF2AEECF43
:102DB000F6FF000EEF22EECFF7FFEF22EECFF8FF87
:102DC0001200040EDBCFE6FF130EDB50E552E75C8A
:102DD0009ADFDB5004DF060EDB501200090EDB50D9
:102DE0000A0DF350DF24D00FE76E090EE7CFDBFFAB
:102DF000D9EF15F0DB50F36E050E07EF16F0F70E66
:102E0000DBCF14F0F80EDBCF15F01200DFCFE6FFBA
:102E1000E3EF15F028DF030EECDE88EF16F035EC5B
:102E200011F0E552E552E552E55200091200BDDE0F
:102E3000EE50EFCFEAFFE96E010E1200130EDB50E9
:102E4000F36E040E07EF16F0040EDB50F36E090E5E
:102E500007EF16F0DBCFE6FFE3EF15F0E76E050EA8
:102E6000E7CFDBFF12008BDF06EF17F0DBCFE6FFCB
:102E700086DF0FEF17F0D950F90FE96EFF0ED4EF90
:0C2E800016F0E96E000EDA20EA6E120077
:042E8C0004012051CC
:102E90001F0B010801E05BD02051600BE842E842C3
:102EA000E842E842E842010801E051D0245103E041
:102EB000240501E04CD02151230A48E0010A40E0FA
:102EC000030A30E0010A25E0240A22E0070A1FE095
:102ED000010A1CE0030A11E0010A01E038D00201F6
:102EE000030EF76F0201E40EF86F020EF96F000196
:102EF000FD930201080EFC6F2AD00201030EF76F4A
:102F00000201E40EFA6F020EFB6F21D020D01FD019
:102F10001ED00201030EF76F0201D90EFA6F020EE6
:102F2000FB6F15D00201030EF76F0201D90EF86F87
:102F3000020EF96F0001FD930201070EFC6F07D02E
:102F40000201030EF76F22C4E0F201D000D012009C
:102F50000201D96BC20EDA6F010EDB6FDC6BDD6B29
:102F6000DE6B080EDF6FD26BD16B1A0E726E1E0E07
:102F7000736E0401000E166F050E176F400E146F6E
:102F80000401196F080E1A6F050E1B6F880E186F5B
:102F90000401480E1E6F050E1F6F400E1C6F1200BD
:102FA000D9CFE6FFE1CFD9FF0201D16B040118BFF1
:102FB00030D0FC0EDBCF14F01951D880145403E24A
:102FC000FC0E19C4DBFF0201D16BFC0EDB50D15D9E
:102FD00019E2D151EA6A080FE96E050EEA22EF50B4
:102FE000E66ED151E76EFD0EDBCFE9FFFE0EDBCFC3
:102FF000EAFFE750E926000EEA22E552E750EF6EBD
:10300000D12BE3D70401400E196F1817187D880ED5
:1030100018130201D15100D0E552E7CFD9FF1200B9
:10302000D9CFE6FFE1CFD9FFE6520201D25101E04C
:1030300030D0DF6ADF2ADF50146E156A145002E1C7
:10304000010E151801E10BD0FD0EDBCFE9FFDB2AE5
:10305000FE0EDBCFEAFF01E3DB2AEF50EBE1DF50AE
:10306000146E156AD950FD0FE96EFF0EDA20EA6E74
:103070001450EE5E1550ED5ADF06FD0EDBCFD3F295
:10308000FE0EDBCFD4F2DFCFD7F20201D86B010EF8
:10309000D26FE552E552E7CFD9FF1200D9CFE6FF54
:1030A000E1CFD9FFE6520201D25101E031D0DF6A0F
:1030B000DF2ADF50146E156AFF0E141801E1155057
:1030C00001E10CD0FD0EDBCFF6FFDB2AFE0EDBCFDD
:1030D000F7FF01E3DB2A0800F550EAE1DF50146E48
:1030E000156AD950FD0FE96EFF0EDA20EA6E145012
:1030F000EE5E1550ED5ADF06FD0EDBCFD3F2FE0E6D
:10310000DBCFD4F2DFCFD7F20201010ED86FD26F3E
:10311000E552E552E7CFD9FF1200D9CFE6FFE1CF64
:10312000D9FFE65204011CBF6BD0030E0201D25D31
:1031300001E1D26BD25101E163D0020ED25D06E112
:1031400004011D6B0201030ED26F54D0D20552E16F
:10315000400E146E156AD751145C000E155803E228
:10316000400EDF6E02D0D7C2DFFFDFCF1DF4DF508D
:10317000D75DD76F480ED56F050ED66FD80515E110
:10318000DF5012E0D3C2F6FFD4C2F7FF0800F550BB
:10319000D5C2E9FFD6C2EAFFEF6ED52B000ED623CB
:1031A000D32BD423DF06ECD713D0DF5011E0D3C2EA
:1031B000E9FFD4C2EAFFEF50D5C2E9FFD6C2EAFF69
:1031C000EF6ED52B000ED623D32BD423DF06EDD7FD
:1031D000D75110E104011D51146E156A400E1418E8
:1031E00001E1155004E10201020ED26F03D0020189
:1031F000030ED26F400E04011C171C7D880E1C1399
:0A320000E552E552E7CFD9FF1200B6
:06320A0004012051600BDD
:10321000E842E842E842E842E842000901E055D0CD
:103220002151070A51E00B0A4FE0070A40E0010A6A
:103230002CE00B0A28E0020A26E0030A22E0080A32
:1032400012E0010A0EE00F0A0AE0030A01E03CD096
:103250000201010EF76F0001040EFC6F36D036D864
:1032600034D090D832D00201010EF76F0201FE0E69
:10327000F86F000EF96F0001FD930201010EFC6F63
:1032800024D0A8D822D0F4D820D00201010EF76FA4
:10329000040124510201F86FF96BFF0EF827000EAC
:1032A000F9230001FD930201010EFC6F0ED0020113
:1032B000010EF76F04012451EA6AFF0FE96E000E58
:1032C000EA2222C4EFFF01D000D01200800E0401D8
:1032D000205D57E12351030A34E0010A10E0030A9C
:1032E00001E04DD00201010EF76F0201740EF86F7C
:1032F0003A0EF96F120E0201FC6FFD6B40D0020115
:10330000010EF76F04012251F66EF76AD890F63677
:10331000F736350EF6263B0EF7220900F5CFF8F208
:103320000A00F5CFF9F2020E0201F76AF825F66EEF
:10333000F951F7220900F5CFFCF20A00F5CFFDF2B2
:103340001ED00201010EF76F04012251F66EF76ADA
:10335000D890F636F736390EF6263B0EF7220900DE
:10336000F5CFF8F20A00F5CFF9F2F8C2F6FFF9C28C
:10337000F7FF0800F5500201FC6FFD6B00D0000163
:10338000FD8312000201010EF76F0F0EE66E710E43
:10339000E66E0F0EE66EAFEC1CF0E552E552E5521C
:1033A000010EE66EFF0EE66E000EE66EAFEC1CF050
:1033B000E552E552E55222C4FEF00401225104E137
:1033C0000001050EFC6F05D00001060EFC6FA8EC95
:1033D00017F012000401286B296B040120511F0B08
:1033E000020A14E0030A0EE0010A01E033D00201F0
:1033F000010EF76F040128810001FDA102D0040134
:10340000288328D00201010EF76F24D00201010E9B
:10341000F76F040124510F0B080DF350156A000FCC
:10342000146E040E15222451800B01E0010E040DD0
:10343000F35002011424FA6F000E1520FB6FFAC23C
:10344000E9FFFBC2EAFFEF50040B03E00401010EA9
:10345000286F00D00201F7050AE10201280EF86F7B
:10346000040EF96F0001FD930201020EFC6F1200C1
:103470000401220510E120511F0B00090CE102019B
:10348000010EF76F030E0401215D03E10001FD81D0
:1034900002D00001FD91040122513AE120511F0B9D
:1034A000020836E124510F0B000932E00201010E3F
:1034B000F76F040124510F0B080DF350156A000F2C
:1034C000146E040E15222451800B01E0010E040D30
:1034D000F35002011424FA6F000E1520FB6F030E47
:1034E0000401215D07E1840EFAC2E9FFFBC2EAFF95
:1034F000EF6E0ED024AF06D0FAC2E9FFFBC2EAFF9E
:10350000EF6A06D0880EFAC2E9FFFBC2EAFFEF6E4F
:023510001200A7
:0E3512006C5002E0000E01D0010E00090BE02B
:10352000040100513C0BE842E8420D0802E10CD8CE
:1035300001D040D808D06C5002E0000E01D0010E3E
:10354000040901E047D81200D9CFE6FFE1CFD9FF47
:10355000E6520201F66BF76BFC6BFD6B05EC19F0A4
:10356000DF6ADF50146E156A010E145C000E1558E8
:103570001BE20201F75101E017D0F76ADF34FE0BBE
:10358000F736F66E3F0EF6263B0EF7220900F5CF12
:1035900014F00800F5CF15F004D015C0FAFF145050
:1035A000F96EFBDFDF2ADDD7DDD8E552E552E7CF44
:1035B000D9FF1200020E0201F65D0AE196D804015D
:1035C00000BD03D0C80E006F02D0880E006F01D07E
:1035D0000FD91200040E0001FC5D0AE122C46EFF47
:1035E0006E50000803E2050EFC6F02D0030EFC6F64
:1035F0000201F6050AE10BD8040104BD03D0C80E90
:10360000046F02D0880E046F01D0F2D81200D9CF17
:10361000E6FFE1CFD9FF020EE1260201080EFC5DB4
:10362000000EFD5905E2FCC2DEFFFDC2DDFF03D046
:10363000080EDE6EDD6A040104930491010EDB5076
:103640000413DFCF05F4000EDB500201FC5F010E16
:10365000DB50FD5B280EFA6F040EFB6F0001FDA32B
:103660001ED0D9CFE9FFDACFEAFFEE50ED1016E019
:10367000F8C2F6FFF9C2F7FF0800F550FAC2E9FFF9
:10368000FBC2EAFFEF6E0201FA2B000EFB23F82BC0
:10369000F923DF06010E01E2DB06E3D71CD0D9CF08
:1036A000E9FFDACFEAFFEE50ED1015E0F8C2E9FFCE
:1036B000F9C2EAFFEF50FAC2E9FFFBC2EAFFEF6E80
:1036C0000201FA2B000EFB23F82BF923DF06010E73
:1036D00001E2DB06E4D7020EE15C02E2E16AE552B8
:1036E000E16EE552E7CFD9FF1200D9CFE6FFE1CF77
:1036F000D9FF020EE126030E04010015E76E010E4C
:10370000E7CFDBFF01C4DFFFDE500201FC27DD5005
:10371000FD23280EF86F040EF96FD9CFE9FFDACF39
:10372000EAFFEE50ED1014E0F8C2E9FFF9C2EAFF3B
:10373000EF50FAC2E9FFFBC2EAFFEF6EFA2B000E70
:10374000FB23F82BF923DF06010E01E2DB06E5D7A8
:10375000020EE15C02E2E16AE552E16EE552E7CF7A
:10376000D9FF12000201F7510CE10401080E016FAC
:10377000200E026F040E036F840E006F0401046FAD
:1037800035D0040120AF22D00201FC510401265D96
:103790000201FD510401275904E226C4FCF227C4AA
:1037A000FDF235DF0201010EF66F0401080E016F14
:1037B000200E026F040E036F800E006F0401280EAE
:1037C000066F040E076FC80E046F10D00201020EC0
:1037D000F66F0401056BC80E046F0401080E016F3B
:1037E000280E026F040E036FC80E006F6D98120052
:1037F0000201F66B0401080E016F200E026F040E29
:0C380000036F880E006F0401046B1200BF
:04380C006DA60FD8BE
:1038100002D06DB613D80001FC0508E16DBA06D0E0
:10382000686A696A69806988020EFC6F12006D6AB5
:10383000696A6D860001010EFC6F12006D6A696A8B
:103840000001FC6B12001EEF1CF00001FC5101E1B5
:103850003AD06850040B04E06950040B01E03CD8F6
:103860006DB231D06850010B04E06950010B01E0EA
:1038700054D86850100B04E06950100B01E024D8B4
:103880006850400B04E06950400B01E03BD86850A1
:10389000200B04E06950200B01E036D86850020B81
:1038A00004E06950020B01E036D8030E0001FC5D14
:1038B00001E209D06850080B06E06950080B03E0EC
:1038C00089EC1AF068961200698468986D82A19A52
:1038D000A08A0300A09A12006D9269946894120065
:1038E0000001FDA10ED0F8DF6D840201080EFE6F0D
:1038F000070EFF6FFE07000EFF5BFE51FF11FAE19E
:103900006D941200689C120070A003D0F8EC1BF0BC
:103910007090689A1200689212006A6A686A9F0E34
:103920006B6E7B0E696E6E6A0F0EE66E710EE66E42
:103930000F0EE66E14D8E552E552E552160E706E83
:1039400068A602D06896FCD76D98F8EC1BF00001D1
:10395000FD910001FE6B0001030EFC6F1200D9CF38
:10396000E6FFE1CFD9FFFD0EDBCFE9FFFE0EDBCF97
:10397000EAFFFC0EDB5004E0EE6AFC0EDB06F9D732
:08398000E552E7CFD9FF120068
:0839880009C013F008C012F0A1
:1039900007C011F007500C02F4CF05F0F3CF04F08C
:1039A00008500D02F4CF07F0F3CF06F00C02F350ED
:1039B0000526F4500622E86A072211500D02F35042
:1039C0000526F4500622E86A072209500C02F3503B
:1039D0000626F450072209500D02086AE86A0822F8
:1039E000F3500726F450082211500E02F350062619
:1039F000F4500722096AE86A0822092212500E02CE
:103A0000F3500726F4500822E86A092213500E02E8
:103A1000F3500826F4500922000C09C013F008C026
:103A200012F008500D02F4CF07F0F3CF06F0095062
:103A30000E02F4CF09F0F3CF08F00D02F350072681
:103A4000F4500822E86A092212500E02F3500726A9
:103A5000F4500822E86A09220EAE33EF1DF012502E
:103A6000085E1350095A13AE000C0D50085E0E503C
:043A7000095A000CE3
:0C3A74001201000202000008D8040A0041
:103A80000000010200010902430002010080320926
:103A900004000001020201000524001001042402B8
:103AA0000205240600010524010001070582030820
:103AB000000209040100020A000000070503024099
:103AC0000000070583024000000403090434034D8D
:103AD000006900630072006F006300680069007095
:103AE00000200054006500630068006E006F006CE9
:103AF000006F0067007900200049006E0063002E0F
:103B00000034034300440043002000520053002DC2
:103B100000320033003200200045006D0075006C5B
:103B2000006100740069006F006E002000440065B1
:103B3000006D006F00863A863AC93ACD3A013B8C57
:013B40002E56
:0E3B4200D9CFE6FFDACFE6FFE1CFD9FFE2CF21
:103B5000DAFFE652E652E652E652D950F90F146EF9
:103B6000FF0EDA20156E020E14C0DBFF030E15C027
:103B7000DBFF020EDBCFE6FF030EDBCFE6FFF90E25
:103B8000DBCFE6FFFA0EDBCFE6FFFB0EDBCFE6FF77
:103B9000D950FC0FE66EFF0EDA20E66E4BEC11F00A
:103BA000146E070EE15C02E2E16AE552E16E145028
:103BB000F3CFDEFFF4CFDDFFFC0EDBCFE9FFFD0E20
:103BC000DBCFEAFFEF6ADECF14F0DDCF15F014C0D3
:103BD000F3FF15C0F4FF040EE15C02E2E16AE55276
:0E3BE000E16EE552E5CFDAFFE7CFD9FF120024
:023BEE002A0E9D
:103BF000F66E080EF76E000EF86E00010900F55023
:103C0000F76F0900F550F86F03E1F76701D03DD079
:103C10000900F550F26F0900F550F36F0900F550F7
:103C2000F46F09000900F550E96E0900F550EA6EDD
:103C3000090009000900F550F56F0900F550F66F0D
:103C400009000900F6CFF9F0F7CFFAF0F8CFFBF052
:103C5000F2C0F6FFF3C0F7FFF4C0F8FF0001F55320
:103C600002E1F65307E00900F550EE6EF507F8E2C1
:103C7000F607F9D7F9C0F6FFFAC0F7FFFBC0F8FF67
:0C3C80000001F707000EF85BBFD7120030
:043C8C00D9CFE6FFA7
:103C9000DACFE6FFE1CFD9FFE2CFDAFFFB0EDBCFD1
:103CA00014F0FC0EDBCF15F00001800E15141AE1A4
:103CB000FB0EDBCFE9FFFC0EDBCFEAFFEECFF3FF1D
:103CC000EDCFF4FFEE2A000EEF22F3CFE9FFF4CFA1
:103CD000EAFFFD0EDBCFEFFFEF50156AF36E15C064
:103CE000F4FF10D0FB0EDB50FE0806E1FD0EDBCF2B
:103CF000E6FF5FEC1FF005D0FD0EDBCFE6FF8FEC9B
:103D00001FF0E552E552E5CFDAFFE7CFD9FF120009
:103D100006500B02F3CF02F0F4CF03F00C02F35085
:103D20000326000EF420046E06500D02F350042604
:103D3000000EF420056E06500E02F35005260750C3
:103D40000B02F3500326F4500422000E0522075004
:103D50000C02F3500426F450052207500D02F350D4
:103D6000052608500B02F3500426F4500522085093
:103D70000C02F350052609500B02F35005261200E1
:103D8000FE0EE3CFE9FFFF0EE3CFEAFFF36AF46A2A
:103D9000EE5203E0F34AF42AFBD71200FF0EE3CF02
:103DA000F8FFE552FF0EE3CFF7FFE552FF0EE3CF3A
:103DB000F6FFE552E66AE66AE66A0900F55209E0AE
:103DC000FD0EE32A05E1FE0EE32A02E1FF0EE32ADF
:103DD000F4D7FD0EE3CF07F0FE0EE3CF08F0FF0EA1
:063DE000E3CF09F0120020
:0A3DE600056A046A036A026A200EEF
:103DF000E76ED8900636073608360936023603369F
:103E0000043605360B50025C0C5003580D50045814
:103E10000E50055809E30B50025E0C50035A0D502A
:0E3E2000045A0E50055A062AE72EE4D7120067
:023E2E005374CB
:103E3000617475733D25690A0D0050492C25317553
:103E40000A0D004D522C253033750A0D002C2530FB
:103E5000347500492C253033692C253033692C25E5
:063E60003033690A0D0079
:0A3E660005D810D893EC05F0FCD746
:103E700012000F0EC112140E6F6E0001FC6B0001D8
:103E8000FD6B0001FE6B01EF05F006EC1CF06FBE50
:0A3E900002D025EC1CF08DEF18F0B5
:063E9A00F36AF46AFF0E5A
:103EA000E124E96EFF0EE220EA6EED6607D02F0EE8
:0E3EB000EF6404D03A0EEF6001D0F32A120046
:023EBE00FF0EF5
:103EC000E350ACBA04D0AF6AAB8EAC8A949CACA27F
:0A3ED000FED7AD6EF36EF46A120027
:063EDA0055425720465737
:103EE00020442056657273696F6E20312E332E3058
:033EF0000A0D00B8
:0C3EF40013EE00F023EE00F0F86A019CD1
:0C3F0000F7EC1DF033EC1FF0FDD71200B1
:043F0C0030313233EB
:0D3F10003435363738396162636465660008
:023F1E0012008F
:0A3F20000000000041000000000056
:00000001FF
